:100000000C945C000C946D050C949A050C9484007F
:100010000C9484000C9484000C9484000C94840050
:100020000C9484000C9484000C9484000C94840040
:100030000C9484000C9484000C9484000C94840030
:100040000C94C7050C9484000C94F9070C9484005C
:100050000C9484000C9484000C9484000C94840010
:100060000C9484000C948400000024272A000025AE
:10007000282B000023262904040404040404040299
:100080000202020202030303030303010204081035
:100090002040800102040810200102040810200002
:1000A0000000070002010000030406000000000039
:1000B00000000000F401830411241FBECFEFD4E040
:1000C000DEBFCDBF11E0A0E0B1E0E2E8F1E102C0A7
:1000D00005900D92A232B107D9F711E0A2E2B1E08A
:1000E00001C01D92A73FB107E1F710E0C8EBD0E0D7
:1000F00004C02297FE010E94BB08C43BD107C9F788
:100100000E947C040C94BF080C940000FC01108237
:100110008FEF81831382128282E2848386E9858352
:10012000178216820895EF92FF920F931F93CF9339
:10013000DF93EC019B0177FF03C020E030E005C0B6
:10014000653B710514F024EB30E02983EC806D8170
:1001500070E06E197109882777FD8095982F982F88
:10016000872F762F662730E040E050E00E94360867
:1001700024EB30E040E050E00E948A08FF2400E0D9
:1001800010E0102F0F2DFE2CEE24E20EF31E041FA4
:10019000151FC801B70120E430E040E050E00E94A4
:1001A0008A083B832A83DF91CF911F910F91FF90A3
:1001B000EF9008955F926F927F928F929F92AF928D
:1001C000BF92CF92DF92EF92FF920F931F93DF9334
:1001D000CF93CDB7DEB76DB67EB6ADB65EB60E9434
:1001E000370620912401309125014091260150913C
:1001F0002701621773078407950750F02C5E3F4F65
:100200004F4F5F4F621773078407950708F4AFC01D
:100210006093240170932501809326019093270118
:10022000E0912201F0912301BB2408C082819381D7
:10023000892B09F0B3940680F781E02D3097B1F750
:10024000BB2009F494C08B2D90E0880F991F2DB727
:100250003EB7281B390B0FB6F8943EBF0FBE2DBF1B
:10026000CDB6DEB60894C11CD11CA0912201B0917C
:10027000230120E013C012968D919C911397892B36
:1002800049F0E22FF0E0EE0FFF1FEC0DFD1DB183F2
:10029000A0832F5F16960D90BC91A02D109759F753
:1002A0002CC0812F90E07C01EE0CFF1CEC0CFD1C9F
:1002B000D7016D917C91FC013197EE0FFF1FEC0D82
:1002C000FD1D40815181DB0112962D913C911397C8
:1002D000DA0112968D919C9113972817390730F403
:1002E000D7014D935C937183608301E01F5F1B1501
:1002F000C0F2002311F410E011C011E000E0F7CFCC
:10030000E12FF0E0EE0FFF1FEC0DFD1D0190F081DD
:10031000E02D61E080810E943D071F5F1B1580F387
:10032000F6B4EE2400E010E08F2C99241EC0EE2DD0
:10033000F0E0EE0FFF1FEC0DFD1D0190F081E02DB0
:1003400022813381280D391D86B58F1510F4005098
:100350001F4FF82EC8018F0D911D28173907A0F7E0
:1003600060E080810E943D07E394EB1400F38A2D46
:10037000952D9C010FB6F8943EBF0FBE2DBF0FB652
:10038000F8947EBE0FBE6DBECF91DF911F910F918D
:10039000FF90EF90DF90CF90BF90AF909F908F90A5
:1003A0007F906F905F9008950F931F938C01FC01D5
:1003B00060838FEF8183138212828091220190915A
:1003C000230197838683109323010093220160E029
:1003D00080810E943D0761E0F80180810E941F0733
:1003E00081E01F910F91089588E291E00E948600BC
:1003F00080E391E00E94860088E391E00E948600FD
:100400000895BC0180E391E00E9493000895BC012F
:1004100088E291E00E9493000895EF92FF920F937B
:100420001F93CF93DF930E94DA0081E691E00E9450
:100430009104882309F416C181E691E00E948E049C
:10044000482F80934C01803F29F410925C01109258
:100450005B0106C081E090E090935C0180935B01BA
:1004600060915B0170915C016130710509F0FAC027
:10047000242F30E0E90194E0D595C7959A95E1F7EE
:100480008091420190914301C817D90709F0EAC051
:100490008091590190915A012F703070019709F0A5
:1004A000D0C010925A011092590130935E012093EE
:1004B0005D01809108010E94A90660E470E00E943D
:1004C000550884E0CC0FDD1F8A95E1F7C62BD72BAA
:1004D000AE01662757FD6095762F20E030E081E67B
:1004E00091E00E94580580915F01909160018330F6
:1004F000910509F44AC0843091054CF4813091058E
:1005000059F182309105ECF5892B89F0ABC085302B
:10051000910509F455C0853091050CF44DC0863025
:10052000910509F474C0079709F09CC07CC060E095
:10053000809114010E943D0720915D0130915E0180
:10054000C901880F991F820F931F880F991F880F69
:10055000991F0E94010286C060E0809114010E94F0
:100560003D0720915D0130915E01C901880F991FFF
:10057000820F931F880F991F880F991F0E940702EF
:1005800071C061E08091040157C060E08091140166
:100590000E943D0780915D0190915E01BC01660F54
:1005A000771F680F791F660F771F660F771F88E325
:1005B00091E00E94930056C061E0809112013CC01E
:1005C00020915D0130915E0121303105A9F484E66E
:1005D00090E09093560180935501309358012093F9
:1005E00057010E9437066093510170935201809326
:1005F00053019093540136C0109258011092570144
:1006000060E070E0809102010E94C7062BC08091DB
:100610005D0190915E01019711F461E001C060E01D
:100620008091000109C080915D0190915E01019768
:1006300031F461E0809110010E943D0713C060E039
:10064000F9CF3093600120935F0170935A0160935A
:10065000590150E060E070E020E030E081E691E098
:100660000E9458050E9437069B01AC0160934D0122
:1006700070934E0180934F019093500180915701E8
:1006800090915801019709F053C0809151019091C8
:100690005201A0915301B0915401281B390B4A0B10
:1006A0005B0B8091550190915601AA2797FDA0956B
:1006B000BA2F281739074A075B07A0F16FEF70E0E0
:1006C000809102010E94C706E0904D01F0904E011A
:1006D00000914F0110915001809151019091520170
:1006E000A0915301B0915401A8019701281B390B27
:1006F0004A0B5B0B8091550190915601880F991F11
:10070000AA2797FDA095BA2F281739074A075B0734
:1007100078F0E0925101F09252010093530110934E
:10072000540106C060E070E0809102010E94C7069B
:10073000DF91CF911F910F91FF90EF90089540E0CE
:100740005BE460E070E081E691E00E94940464E67E
:1007500070E080E090E00E94450660E070E08091EB
:1007600002010E94C706609116017091170188E28C
:1007700091E00E94D401609118017091190180E309
:1007800091E00E94D401609106017091070188E315
:1007900091E00E94D40161E0809114010E943D0724
:1007A0006DE570E088E391E00E94930061E0809144
:1007B00000010E941F0761E0809102010E941F0753
:1007C00061E0809104010E941F0760E08EE00E94BA
:1007D0001F0760E08FE00E941F0760E080E10E9439
:1007E0001F0760E081E10E941F0761E08EE00E9428
:1007F0003D0761E08FE00E943D0761E080E10E94DB
:100800003D0761E081E10E943D07809140010E9427
:10081000A906815092403CF081E090E09093450120
:100820008093440104C010924501109244018091CC
:100830000A010E94A906815092403CF082E090E0BB
:10084000909347018093460104C010924701109293
:10085000460180910C010E94A906815092403CF013
:1008600084E090E0909349018093480104C0109285
:1008700049011092480180910E010E94A906815001
:1008800092403CF088E090E090934B0180934A01C5
:1008900004C010924B0110924A0180914601909140
:1008A00047012091440130914501820F931F20910F
:1008B000480130914901820F931F20914A013091E4
:1008C0004B01820F931F909343018093420160E09C
:1008D000809104010E943D0761E0809114010E9413
:1008E0003D0760E0809110010E943D0760E080912B
:1008F00012010E943D0708950E946F060E949F0307
:100900000E940D02FDCF8FE191E0909362018093F0
:1009100061010895862F0E94C10708950E94DA0799
:1009200008950E94C9070895CB01BA010E94880763
:1009300008952F923F924F925F926F927F928F9283
:100940009F92AF92BF92CF92DF92EF92FF920F935E
:100950001F93DF93CF93CDB7DEB7A0970FB6F89470
:10096000DEBF0FBECDBF1C016A017B0141155105E1
:100970006105710549F4DC01ED91FC910190F08174
:10098000E02D60E3099554C0882499245401422E37
:1009900055246624772401E010E00C0F1D1F080D7C
:1009A000191DC701B601A30192010E946808F80150
:1009B00060830894811C911CA11CB11CC701B60165
:1009C000A30192010E946808C901DA016C017D014E
:1009D000C114D104E104F104F1F681E0E82EF12C18
:1009E000EC0EFD1EE80CF91C3E010894611C711C04
:1009F000D501C4010197A109B1096C01C818D90832
:100A000014C0F601EE0DFF1D60816A3010F4605DC8
:100A100001C0695CD101ED91FC910190F081E02D64
:100A2000C10109950894E108F1086E147F0449F7A3
:100A3000A0960FB6F894DEBF0FBECDBFCF91DF9169
:100A40001F910F91FF90EF90DF90CF90BF90AF90EC
:100A50009F908F907F906F905F904F903F902F90DE
:100A60000895EF92FF920F931F93CF93DF93EC01C2
:100A70007A018B0177FF0FC0E881F9810190F08145
:100A8000E02D6DE2099510950095F094E094E11C3D
:100A9000F11C011D111D2AE0B801A701CE010E9421
:100AA0009904DF91CF911F910F91FF90EF900895DE
:100AB000DC012115310541F4ED91FC910190F081AB
:100AC000E02D642F099508952A30310519F40E940C
:100AD000310508950E94990408951F920F920FB650
:100AE0000F9211242F933F934F935F936F937F93B4
:100AF0008F939F93AF93BF93EF93FF938091630185
:100B000090916401892B29F0E0916301F0916401D7
:100B10000995FF91EF91BF91AF919F918F917F9137
:100B20006F915F914F913F912F910F900FBE0F905A
:100B30001F9018951F920F920FB60F9211242F93AA
:100B40003F934F935F936F937F938F939F93AF9355
:100B5000BF93EF93FF938091650190916601892B7C
:100B600029F0E0916501F09166010995FF91EF91FF
:100B7000BF91AF919F918F917F916F915F914F91B5
:100B80003F912F910F900FBE0F901F9018951F92BD
:100B90000F920FB60F9211242F938F939F93AF93C1
:100BA000BF938091670190916801A0916901B09114
:100BB0006A010196A11DB11D8093670190936801A0
:100BC000A0936901B0936A0180916B0190916C01CF
:100BD000A0916D01B0916E018050904CAF4FBF4F0E
:100BE00080936B0190936C01A0936D01B0936E01A3
:100BF00027C080916B0190916C01A0916D01B09123
:100C00006E0180589E43A040B04080936B0190934A
:100C10006C01A0936D01B0936E0180916F01909172
:100C20007001A0917101B09172010196A11DB11DD9
:100C300080936F0190937001A0937101B093720142
:100C400080916B0190916C01A0916D01B0916E014A
:100C500081589E43A040B04060F6BF91AF919F91F4
:100C60008F912F910F900FBE0F901F9018958FB7F7
:100C7000F89420916F013091700140917101509171
:100C800072018FBFB901CA010895EF92FF920F93CD
:100C90001F937B018C018FB7F89440916F015091A5
:100CA000700160917101709172018FBF2FB7F8943C
:100CB00080916F0190917001A0917101B0917201CA
:100CC0002FBF841B950BA60BB70BE816F9060A0776
:100CD0001B0760F71F910F91FF90EF900895789494
:100CE00084B5826084BD84B5816084BD85B5826031
:100CF00085BD85B5816085BDEEE6F0E080818160CF
:100D00008083E1E8F0E0808182608083808181607F
:100D10008083E0E8F0E0808181608083E1EBF0E0B7
:100D2000808184608083E0EBF0E08081816080835B
:100D3000EAE7F0E080818460808380818260808344
:100D40008081816080838081806880831092C1006F
:100D500008958F7090911A019295990F990F907C38
:100D6000982B90937C0080917A00806480937A0025
:100D700080917A0086FDFCCF209178004091790027
:100D8000942F80E030E0282B392BC90108951F9360
:100D9000CF93DF93182FEB0161E00E941F07E12F33
:100DA000F0E0E156FF4F8491833051F48091800050
:100DB000806880938000D0938900C09388003BC0F6
:100DC000843051F480918000806280938000D093C1
:100DD0008B00C0938A002FC0813039F4209729F10D
:100DE00084B5806884BDC7BD26C0823039F42097A1
:100DF000E1F084B5806284BDC8BD1DC0863041F479
:100E00008091B00080688093B000C093B30013C09D
:100E1000873041F48091B00080628093B000C0932D
:100E2000B40009C0C038D10514F460E001C061E02D
:100E3000812F0E943D07DF91CF911F910895282FA8
:100E400030E0C90185579F4FFC01949129583F4FCD
:100E5000F9018491882381F0E82FF0E0E859FF4FF1
:100E6000E491F0E0662329F48081909589238083C2
:100E700008958081892B80830895482F50E0CA010E
:100E800081569F4FFC012491CA0185579F4FFC0159
:100E9000949149585F4FFA0134913323C1F12223D1
:100EA00031F1233021F4809180008F7705C0243008
:100EB00031F4809180008F7D8093800018C02130B4
:100EC00019F484B58F7704C0223021F484B58F7D66
:100ED00084BD0DC0263021F48091B0008F7705C00D
:100EE000273029F48091B0008F7D8093B000E32FEC
:100EF000F0E0E359FF4FE491F0E0662329F48081AC
:100F000090958923808308958081892B808308951B
:100F1000EF92FF920F931F937B018C0122E030E050
:100F200040E050E00E948A08205C3D4B404F5F4FFC
:100F3000CA01B901A80197010E948A08C901DA0112
:100F40000197A109B109292F3A2F4B2F552747FDAA
:100F50005A950196A11DB11D2093C5008150809323
:100F6000C400E1ECF0E08081806180838081886052
:100F700080838081806880831F910F91FF90EF9024
:100F80000895982F8091C00085FFFCCF9093C600F4
:100F90000895809173019091740180589F4F209122
:100FA000750130917601821B930B60E870E00E941E
:100FB0005508089540917501509176018091730113
:100FC000909174018417950719F42FEF3FEF0FC02C
:100FD000FA01E958FE4F2081CA01019660E870E0ED
:100FE0000E945508909376018093750130E0C90105
:100FF00008951F920F920FB60F9211242F933F93D3
:101000004F935F936F937F938F939F93AF93BF9310
:10101000EF93FF934091C600E0917301F09174014A
:10102000CF01019660E870E00E9455089C01809114
:101030007501909176012817390739F0E958FE4F6C
:1010400040833093740120937301FF91EF91BF911E
:10105000AF919F918F917F916F915F914F913F9150
:101060002F910F900FBE0F901F901895629FD00187
:10107000739FF001829FE00DF11D649FE00DF11D53
:10108000929FF00D839FF00D749FF00D659FF00D02
:101090009927729FB00DE11DF91F639FB00DE11DEF
:1010A000F91FBD01CF011124089597FB092E0726D2
:1010B0000AD077FD04D049D006D000201AF47095EC
:1010C00061957F4F0895F6F7909581959F4F08950C
:1010D000A1E21A2EAA1BBB1BFD010DC0AA1FBB1F3C
:1010E000EE1FFF1FA217B307E407F50720F0A21BAE
:1010F000B30BE40BF50B661F771F881F991F1A941B
:1011000069F760957095809590959B01AC01BD0144
:10111000CF01089597FB092E05260ED057FD04D068
:10112000D7DF0AD0001C38F45095409530952195B2
:101130003F4F4F4F5F4F0895F6F79095809570950C
:1011400061957F4F8F4F9F4F0895AA1BBB1B51E1A5
:1011500007C0AA1FBB1FA617B70710F0A61BB70B27
:10116000881F991F5A95A9F780959095BC01CD01CC
:101170000895EE0FFF1F0590F491E02D0994F89467
:02118000FFCF9F
:1011820008000B000400020004000100020003003A
:1011920003000500070009000A0001000000008AA0
:0211A200040047
:00000001FF
